:0835470033302E31202020005A
:10300F00C103C10542029C00044402660000000097
:10301F0044026A0000000044026E000000004402F7
:10302F0072000000004402760000000044027A00A3
:10303F0000000044027E00000000440282000000F5
:06304F0000420286000AA7
:10348900758850758922758E0C758AAE758CAE75E6
:063499008BC7758DC722F0
:10349F0075F1FEE4F5F2F5F375A41A75D41175E123
:0534AF000675E2C022D9
:1034C50075D10275BC4075E8C075BA1F43E6082280
:0C34FC0075A14075F80175A202D2AE2245
:0435770075B2832284
:0B35080075CA8275CBFDD2CAD2AD227D
:0D34D5007592077593F875910443E6802207
:10344200E4F5D912357712349F1234C51234FC12C6
:0834520034891235080234D55B
:0B351300E5B030E403C20622D206221D
:081A2400E4FFE5B030E3010F1F
:011A2C002297
:1032D200EF25E0FFA206E4334F14601314600A14D2
:1032E200600A240370097F36227F37227F35227FCE
:0232F200342284
:101DAF00E4FDFF1215437D017F011215437D027F74
:101DBF00021215437D037F031215437D0A7F041220
:101DCF0015437D0B7F051215437D0C7F06121543BE
:101DDF007D0D7F071215437D0E7F081215437D0F72
:101DEF007F09121543D3E5139430E5129403400B8A
:101DFF0090028EE4F0A37410F08046D3E513946440
:101E0F00E5129402400B90028EE4F0A37408F08068
:101E1F0030D3E5139498E5129401400B90028EE4B1
:101E2F00F0A37404F0801AD3E51394CCE512940058
:101E3F0090028EE44007F0A37402F08004F0A30434
:101E4F00F0D3E50F9430E50E9403400B900290E42D
:101E5F00F0A37410F08046D3E50F9464E50E94025E
:101E6F00400B900290E4F0A37408F08030D3E50F9C
:101E7F009498E50E9401400B900290E4F0A3740443
:101E8F00F0801AD3E50F94CCE50E9400900290E405
:101E9F004007F0A37402F08004F0A304F0D3E50B25
:101EAF009430E50A9403400B900294E4F0A374D0AD
:101EBF00F08047D3E50B9464E50A9402400B90023F
:101ECF0094E4F0A374C8F08031D3E50B9498E50A3D
:101EDF009401400B900294E4F0A374C4F0801BD3E0
:101EEF00E50B94CCE50A9400900294E44007F0A32C
:101EFF0074C2F08005F0A374C1F0D3E51B9430E5F4
:101F0F001A9403400B900292E4F0A374D0F0804730
:101F1F00D3E51B9464E51A9402400B900292E4F00F
:101F2F00A374C8F08031D3E51B9498E51A9401404F
:101F3F000B900292E4F0A374C4F0801BD3E51B94C2
:101F4F00CCE51A9400900292E44007F0A374C2F01B
:101F5F008005F0A374C1F0E5097003022015D3E5E5
:101F6F00179430E5169403400890029B7410F0808C
:101F7F003CD3E5179464E5169402400890029B74D5
:101F8F0008F08029D3E5179498E51694014008903E
:101F9F00029B7404F08016D3E51794CCE5169400D9
:101FAF0090029B40057402F080037401F0D3E51199
:101FBF009414E5109403400890029BE044A0803BEA
:101FCF00D3E5119454E5109402400890029BE0442D
:101FDF00808028D3E51194A4E51094014008900265
:101FEF009BE044608015D3E51194ECE510940090CC
:101FFF00029BE04004444080024420FF900298E49A
:10200F00F0A3EFF08007E4900298F0A3F0E50870DA
:10201F00030220CAD3E51D9430E51C9403400890B9
:10202F00029B7410F0803CD3E51D9464E51C940270
:10203F00400890029B7408F08029D3E51D9498E521
:10204F001C9401400890029B7404F08016D3E51D88
:10205F0094CCE51C940090029B40057402F0800321
:10206F007401F0D3E5199414E51894034008900215
:10207F009BE044A0803BD3E5199454E518940240AB
:10208F000890029BE044808028D3E51994A4E518BA
:10209F009401400890029BE044608015D3E51994A9
:1020AF00ECE518940090029BE04004444080024409
:1020BF0020FF900296E4F0A3EFF022E4900296F056
:0320CF00A3F02259
:1020D200123442121A247571077523077524D0121F
:1020E20035131232D290029FEFF01234EF43F60111
:1020F20030060543A480C287D2AF12342812323B85
:10210200E56E603914601414600924FE702C6309B2
:102112000180036308011233D6801F30030F30069B
:1021220005A287B39287308711C211800DE4900215
:10213200DAF0123571300602C287E4F56E3005100E
:1021420090029FE0FF7BFF7A35794712306FC2051C
:10215200300713C207E52445236008E524152470DF
:10216200021523121DAF7B017A0279C112320FEFE1
:10217200608E9002C3E0121D5D21F004223705211A
:10218200B214219A1621A71721B71A21D91B21E4CB
:102192001D21EA1E00002287200603022287D28721
:1021A200C211022287200603022287C287022287E7
:1021B200D2030222877B017A0279C19002D1EBF02D
:1021C200A3EAF0A3E9F0121B26FE90029FE0FF6E45
:1021D2006003022287800590029FE0FF12333702DC
:1021E200228712355E02228712356B0222877B011B
:1021F2007A0279C19002D4EBF0A3EAF0A3E9F0905D
:102202000003121B3FFF90029FE06F707830876DD2
:102212009002D404F0A3EAF0A3E9F0900005121BA7
:102222003FFF900006121B3FFD900004121B3FFB74
:1022320012197B80487B017A0279C19002D4EBF0BB
:10224200A3EAF0A3E9F0900003121B3FFF90029F64
:10225200E06F70313087269002D404F0A3EAF0A335
:10226200E9F0900005121B3FFF900006121B3FFD94
:10227200900004121B3FFB122C2D12323B90029F46
:10228200E0FF1233992087030221689002C3E01411
:10229200603424FA60531470030223392406600365
:1022A2000221681234B47B017A0279C19002D1EB27
:1022B200F0A3EAF0A3E9F0900003121B3F9002DAC8
:1022C200F0123571806B1234B47B017A0279C190BD
:1022D20002D1EBF0A3EAF0A3E9F0900003121B3F56
:1022E2009002DAF012323B80481234B47B017A0257
:1022F20079C19002D7EBF0A3EAF0A3E9F0900003D2
:10230200121B3FFF900004121B3FFD900005121BA1
:102312003FFBC0039002D7E0FBA3E0FAA3E0F990F1
:102322000006121B3F90030BF0D003122CE3123273
:102332003B1235330221681234B47B017A0279C12F
:102342009002D7EBF0A3EAF0A3E9F0900003121B8E
:102352003FFF900004121B3FFD900005121B3FFB44
:0C23620012250912323B123533022168AB
:102EA700E5B05407F56D6571600CE56D6571F56FFB
:102EB700757003856D71E57060361570E57070305B
:102EC700E56F30E211E56D20E20C9002647405F0C5
:102ED700A374DCF0D200E56F30E108E56D20E10373
:102EE700756E02E56F30E008E56D20E003756E0151
:102EF700300027900265E024FFF0900264E034FF81
:102F0700F0E5B054046005756E04C200900264E0F9
:0A2F17007002A3E07004C200D205AE
:012F2100228D
:031A12000208A720
:1008A700C0E0C0F0C083C082C0D075D000C000C017
:0D08B70001C002C003C004C005C006C00798
:1008C400C2CF90029AE4F0900288A3E0F5A39002CC
:1008D4009CE4F0A37404F0F5BB75E8D02002030295
:1008E4001528E50D2558FFE50C3557FEE4FCFD9071
:1008F40002A1121D20E515255EFFE514355DFEE419
:10090400FCFD9002A5121D20E47FFF7E03FDFC90F8
:1009140002A1E0F8A3E0F9A3E0FAA3E0FBD3121CE0
:10092400E9400A9002A1121D2C000003FFE47FFF9E
:100934007E03FDFC9002A5E0F8A3E0F9A3E0FAA38E
:10094400E0FBD3121CE9400A9002A5121D2C000002
:1009540003FF9002A1E0F8A3E0F9A3E0FAA3E0FB0F
:10096400C374FF9BFB74039AFAE499F9E498F8AE14
:1009740055AF56E4FCFD121BCC780A121CFAC004D5
:10098400C005C006C007AE59AF5AE4FCFD9002A1F1
:10099400E0F8A3E0F9A3E0FAA3E0FB121BCC780A89
:1009A400121CFAD003D002D001D000EF2BFFEE3A94
:1009B400FEED39FDEC38FC9002A9121D209002A531
:1009C400E0F8A3E0F9A3E0FAA3E0FBC374FF9BFB08
:1009D40074039AFAE499F9E498F8AE5BAF5CE4FC2A
:1009E400FD121BCC780A121CFAC004C005C006C054
:1009F40007AE5FAF60E4FCFD9002A5E0F8A3E0F968
:100A0400A3E0FAA3E0FB121BCC780A121CFAD00371
:100A1400D002D001D000EF2BFFEE3AFEED39FDEC11
:100A240038FC9002AD121D2090026AE0FCA3E0FDA8
:100A3400A3E0FEA3E0FF9002A9E0F8A3E0F9A3E09D
:100A4400FAA3E0FBD3121CE940359002A9E0FCA311
:100A5400E0FDA3E0FEA3E0FF90026A121D209002D5
:100A6400A9E0FCA3E0FDA3E0FEA3E024FCFFEE3438
:100A7400FFFEED34FFFDEC34FFFC900272805290D7
:100A84000272E0FCA3E0FDA3E0FEA3E0FF9002A954
:100A9400E0F8A3E0F9A3E0FAA3E0FBC3121CE950D9
:100AA400339002A9E0FCA3E0FDA3E0FEA3E0FF90E5
:100AB4000272121D209002A9E0FCA3E0FDA3E0FE57
:100AC400A3E02404FFE43EFEE43DFDE43CFC90028C
:100AD4006A121D2090027AE0FCA3E0FDA3E0FEA3CD
:100AE400E0FF9002ADE0F8A3E0F9A3E0FAA3E0FB95
:100AF400D3121CE940359002ADE0FCA3E0FDA3E075
:100B0400FEA3E0FF90027A121D209002ADE0FCA348
:100B1400E0FDA3E0FEA3E024FCFFEE34FFFEED3491
:100B2400FFFDEC34FFFC9002828052900282E0FCD4
:100B3400A3E0FDA3E0FEA3E0FF9002ADE0F8A3E094
:100B4400F9A3E0FAA3E0FBC3121CE950339002AD11
:100B5400E0FCA3E0FDA3E0FEA3E0FF900282121DEF
:100B6400209002ADE0FCA3E0FDA3E0FEA3E024049A
:100B7400FFE43EFEE43DFDE43CFC90027A121D20BD
:100B8400900272E0FCA3E0FDA3E0FEA3E0FF90026C
:100B9400A9121D20900282E0FCA3E0FDA3E0FEA3C5
:100BA400E0FF9002AD121D20E47FFF7E03FDFC9068
:100BB40002A9E0F8A3E0F9A3E0FAA3E0FBD3121C36
:100BC400E9400A9002A9121D2C000003FFE47FFFF4
:100BD4007E03FDFC9002ADE0F8A3E0F9A3E0FAA3E4
:100BE400E0FBD3121CE9400A9002AD121D2C000058
:100BF40003FFE5097003020F03AE53AF54E4FCFD99
:100C04009002A9E0F8A3E0F9A3E0FAA3E0FBC31281
:100C14001CE94003020D2B9002A9E0FCA3E0FDA314
:100C2400E0FEA3E0FF780A121D0D9002B1121D2010
:100C34009002B1E0FCA3E0FDA3E0FEA3E0FFC00648
:100C4400C007AE10AF11AB07AA06E4F9F8D007D07D
:100C540006121C579002B1121D209002B1E0F8A3B5
:100C6400E0F9A3E0FAA3E0FBAE16AF17E4FCFD1233
:100C74001BCC9002B1121D209002B1E0FCA3E0FD58
:100C8400A3E0FEA3E0FF780A121CFA9002B1121D41
:100C9400209002A9E0FCA3E0FDA3E0FEA3E0FF781E
:100CA4000A121D0D9002BD121D209002BDE0FCA38E
:100CB400E0FDA3E0FEA3E0FFC006C007AE10AF1145
:100CC400AB07AA06E4F9F8D007D006121C57900225
:100CD400BD121D20E47FFF7E03FDFC9002BDE0F801
:100CE400A3E0F9A3E0FAA3E0FBC3121CE99002BD60
:100CF4005019E0F8C374FF9BFF74039AFEE499FD56
:100D0400E498FC9002BD121D208007121D2C0000E7
:100D140000009002BDE0F8A3E0F9A3E0FAA3E0FB31
:100D2400AE0EAF0F020EC0AE10AF11E4FCFD900288
:100D3400A9E0F8A3E0F9A3E0FAA3E0FBD3121CE9CD
:100D4400402AAE10AF11AB07AA069002A9E0FCA39B
:100D5400E0FDA3E0FEA3E09BFFEE9AFEED9400FD10
:100D6400EC9400FC9002B1121D20800A9002B11292
:100D74001D2C000000009002B1E0FCA3E0FDA3E004
:100D8400FEA3E0FF780A121D0D9002B1121D20C3CC
:100D9400E51194FFE5109403503BC374FF9511FFD4
:100DA40074039510FEE4FCFD9002BD121D20900218
:100DB400B1E0FCA3E0FDA3E0FEA3E0FF9002BDE0F0
:100DC400F8A3E0F9A3E0FAA3E0FB121C579002B1E8
:100DD400121D20800A9002BD121D2C0000000090FC
:100DE40002B1E0F8A3E0F9A3E0FAA3E0FBAE0AAF96
:100DF4000BE4FCFD121BCC9002B1121D209002B139
:100E0400E0FCA3E0FDA3E0FEA3E0FF780A121CFAD5
:100E14009002B1121D20E47FFF7E03FDFC9002A925
:100E2400E0F8A3E0F9A3E0FAA3E0FBC3121CE95045
:100E34001C9002A9E0F8C374FF9BFF74039AFEE4BC
:100E440099FDE498FC9002BD121D20800A9002BD19
:100E5400121D2C000000009002BDE0FCA3E0FDA3E5
:100E6400E0FEA3E0FF780A121D0D9002BD121D20C2
:100E7400C3E51194FFE5109403502F9002BDE0FCEC
:100E8400A3E0FDA3E0FEA3E0FFC006C007C374FF18
:100E94009511FF74039510AB07FAE4F9F8D007D065
:100EA40006121C579002BD121D209002BDE0F8A34B
:100EB400E0F9A3E0FAA3E0FBAE16AF17E4FCFD12E1
:100EC4001BCC9002BD121D209002BDE0FCA3E0FDEE
:100ED400A3E0FEA3E0FF780A121CFA9002BD121DE3
:100EE400209002B1E0FCA3E0FDA3E0FEA3E0FF90AC
:100EF40002BDE0F8A3E0F9A3E0FAA3E0FB80599077
:100F040002A9E0F8A3E0F9A3E0FAA3E0FBC374FFAD
:100F14009BFB74039AFAE499F9E498F8AE0EAF0FC8
:100F2400E4FCFD121BCC780A121CFAC004C005C0F4
:100F340006C007AE0AAF0BE4FCFD9002A9E0F8A3DB
:100F4400E0F9A3E0FAA3E0FB121BCC780A121CFA26
:100F5400D003D002D001D000EF2BFFEE3AFEED39E2
:100F6400FDEC38FC9002B1121D20E508700302125A
:100F740077AE18AF19E4FCFD9002ADE0F8A3E0F9F8
:100F8400A3E0FAA3E0FBC3121CE940030210A39000
:100F940002ADE0FCA3E0FDA3E0FEA3E0FF780A12AB
:100FA4001D0D9002B5121D209002B5E0FCA3E0FDDA
:100FB400A3E0FEA3E0FFC006C007AE18AF19AB075D
:100FC400AA06E4F9F8D007D006121C579002B5120D
:100FD4001D209002B5E0F8A3E0F9A3E0FAA3E0FB3A
:100FE400AE1CAF1DE4FCFD121BCC9002B5121D20FB
:100FF4009002B5E0FCA3E0FDA3E0FEA3E0FF780AC5
:10100400121CFA9002B5121D209002ADE0FCA3E080
:10101400FDA3E0FEA3E0FF780A121D0D9002B912B1
:101024001D209002B9E0FCA3E0FDA3E0FEA3E0FFD5
:10103400C006C007AE18AF19AB07AA06E4F9F8D08A
:1010440007D006121C579002B9121D20E47FFF7EC0
:1010540003FDFC9002B9E0F8A3E0F9A3E0FAA3E0F1
:10106400FBC3121CE99002B95019E0F8C374FF9B4A
:10107400FF74039AFEE499FDE498FC9002B9121DF2
:10108400208007121D2C000000009002B9E0F8A394
:10109400E0F9A3E0FAA3E0FBAE12AF13021236AEFE
:1010A40018AF19E4FCFD9002ADE0F8A3E0F9A3E069
:1010B400FAA3E0FBD3121CE9402AAE18AF19AB0720
:1010C400AA069002ADE0FCA3E0FDA3E0FEA3E09B32
:1010D400FFEE9AFEED9400FDEC9400FC9002B51234
:1010E4001D20800A9002B5121D2C00000000900201
:1010F400B5E0FCA3E0FDA3E0FEA3E0FF780A121D27
:101104000D9002B5121D20C3E51994FFE518940350
:101114005039C374FF9519FF74039518FEE4FCFD60
:101124009002B9121D209002B5E0FCA3E0FDA3E0FB
:10113400FEA3E0FFA3E0F8A3E0F9A3E0FAA3E0FB39
:10114400121C579002B5121D20800A9002B9121D7C
:101154002C000000009002B5E0F8A3E0F9A3E0FA47
:10116400A3E0FBAE1AAF1BE4FCFD121BCC9002B54E
:10117400121D209002B5E0FCA3E0FDA3E0FEA3E075
:10118400FF780A121CFA9002B5121D20E47FFF7E3C
:1011940003FDFC9002ADE0F8A3E0F9A3E0FAA3E0BC
:1011A400FBC3121CE9501C9002ADE0F8C374FF9B12
:1011B400FF74039AFEE499FDE498FC9002B9121DB1
:1011C40020800A9002B9121D2C000000009002B980
:1011D400E0FCA3E0FDA3E0FEA3E0FF780A121D0DEE
:1011E4009002B9121D20C3E51994FFE51894035029
:1011F4002F9002B9E0FCA3E0FDA3E0FEA3E0FFC052
:1012040006C007C374FF9519FF74039518AB07FA5A
:10121400E4F9F8D007D006121C579002B9121D2029
:101224009002B9E0F8A3E0F9A3E0FAA3E0FBAE1C56
:10123400AF1DE4FCFD121BCC9002B9121D209002DC
:10124400B9E0FCA3E0FDA3E0FEA3E0FF780A121CD2
:10125400FA9002B9121D209002B5E0FCA3E0FDA3B0
:10126400E0FEA3E0FFA3E0F8A3E0F9A3E0FAA3E023
:10127400FB80599002ADE0F8A3E0F9A3E0FAA3E003
:10128400FBC374FF9BFB74039AFAE499F9E498F89E
:10129400AE12AF13E4FCFD121BCC780A121CFAC088
:1012A40004C005C006C007AE1AAF1BE4FCFD9002E3
:1012B400ADE0F8A3E0F9A3E0FAA3E0FB121BCC78BD
:1012C4000A121CFAD003D002D001D000EF2BFFEE9B
:1012D4003AFEED39FDEC38FC9002B5121D20900267
:1012E40066E0FCA3E0FDA3E0FEA3E0FF9002B1E012
:1012F400F8A3E0F9A3E0FAA3E0FBD3121CE940351C
:101304009002B1E0FCA3E0FDA3E0FEA3E0FF9002A5
:1013140066121D209002B1E0FCA3E0FDA3E0FEA351
:10132400E024FCFFEE34FFFEED34FFFDEC34FFFC63
:1013340090026E805290026EE0FCA3E0FDA3E0FEFA
:10134400A3E0FF9002B1E0F8A3E0F9A3E0FAA3E080
:10135400FBC3121CE950339002B1E0FCA3E0FDA3EF
:10136400E0FEA3E0FF90026E121D209002B1E0FCAB
:10137400A3E0FDA3E0FEA3E02404FFE43EFEE43D7D
:10138400FDE43CFC900266121D20900276E0FCA372
:10139400E0FDA3E0FEA3E0FF9002B5E0F8A3E0F9CE
:1013A400A3E0FAA3E0FBD3121CE940359002B5E0B8
:1013B400FCA3E0FDA3E0FEA3E0FF900276121D2053
:1013C4009002B5E0FCA3E0FDA3E0FEA3E024FCFF53
:1013D400EE34FFFEED34FFFDEC34FFFC90027E8022
:1013E4005290027EE0FCA3E0FDA3E0FEA3E0FF90A8
:1013F40002B5E0F8A3E0F9A3E0FAA3E0FBC3121CF2
:10140400E950339002B5E0FCA3E0FDA3E0FEA3E0C5
:10141400FF90027E121D209002B5E0FCA3E0FDA324
:10142400E0FEA3E02404FFE43EFEE43DFDE43CFCD6
:10143400900276121D2090026EE0FCA3E0FDA3E072
:10144400FEA3E0FF9002B1121D2090027EE0FCA3F7
:10145400E0FDA3E0FEA3E0FF9002B5121D20E47FAF
:10146400FF7E03FDFC9002B1E0F8A3E0F9A3E0FAEB
:10147400A3E0FBD3121CE9400A9002B1121D2C0018
:101484000003FFE47FFF7E03FDFC9002B5E0F8A3B8
:10149400E0F9A3E0FAA3E0FBD3121CE9400A9002AE
:1014A400B5121D2C000003FFC2849002B1E0FCA31E
:1014B400E0FDA3E0FEA3E0FF7802121CFA9002888C
:1014C400EEF0A3EFF09002B1A3A3A3E05403FFE472
:1014D400FEFDFC7806121D0DC004C005C006C00741
:1014E400A3E0FCA3E0FDA3E0FEA3E0FF7806121C4A
:1014F400FAD003D002D001D000EF4BFFEE4AFE90A9
:10150400028AEEF0A3EFF09002B5A3A3A3E0543F48
:10151400FFE4FEFDFC7802121D0D90028CEEF0A398
:04152400EFF0C20220
:10152800D007D006D005D004D003D002D001D00017
:0B153800D0D0D082D083D0F0D0E032C1
:031A1500022E237B
:102E2300C0E0C083C082C0D075D000C004C005C05C
:102E330006C007C2FF90029AE004F0C36480948343
:102E43005007E0FF3395E0801F90029AE0FFC364D0
:102E5300809485502B90029EE0FD3395E0FCEF3388
:102E630095E0FEEF2DFFEE3CFEEF25E0FFEE33FE97
:102E730074882FF58274023EF583A3E0F5A38013D3
:102E830090029EE02402F0E0D3648094854002E443
:102E9300F0D284D007D006D005D004D0D0D082D0D1
:042EA30083D0E032C6
:031A2D000233B8C9
:1033B800C0E0C083C082C0D075D000C00753917FE1
:0E33C800122EA7D007D0D0D082D083D0E03212
:031A2100022B276E
:102B2700C0E0C0F0C083C082C0D075D000C000C074
:072B370004C005C006C00741
:102B3E00C2EDAFBEEFFEADBDEDFF90029CE07004A6
:102B4E00A3E06402705EE5BBB403047D0180027DE8
:102B5E0000E5BBB40D047C0180027C00EC4D6035B9
:102B6E00D3EF94C8EE648094834010AFBBEF25E0A2
:102B7E00244DF876030876C8022C18C3EF9468EE3D
:102B8E0064809480500FAFBBEF25E0244DF87600A3
:102B9E000876688075ADBBED25E0244DF8A60608D5
:102BAE00A6078066ADBBED25E0244DF8A60608A667
:102BBE000790029CE475F001121BA0FEC3E5F09491
:102BCE000AEE64809480500990029CA3E0F5BB80CD
:102BDE0036900286E475F001121BA0FED3E5F09448
:102BEE0013EE64809480400B900286E4F0A3740A86
:102BFE00F0D20790029CE4F0A37402F0D20290028D
:0A2C0E0086A3E0540FF5BB75E8D073
:102C1800D007D006D005D004D000D0D0D082D08341
:052C2800D0F0D0E03205
:10305500420262000042020D00004202080000C167
:053065000FC10EC10DBA
:0A352900C20EC20FE490020CF02263
:1032AF00E4900262F0A3F090020DF0A3F0A3F0906F
:1032BF000208F0A3F0900203F0A37440F0E4900230
:0332CF000BF022DF
:061A1B001235290232AF72
:0D34E20075C19043E60190020A7401F022CA
:1034B40043C140E5C120E5FB121A1BE490020AF067
:0134C40022E5
:0A35330053C1BF90020A7401F02298
:0D34EF00AE071234E2900207EEF0021A1B45
:10328A00E49003A7F0A3F0300E02FF22200FFDD234
:10329A000E900205E4F0A37410F0900250EFF0E4EF
:0432AA00A3F07F010D
:0132AE0022FD
:1031DB00300E0A900205E07002A3E070037F00221C
:1031EB00900206E024FFF0900205E034FFF090021D
:1031FB0051E0FE04F074522EF582E43402F583EFB5
:04320B00F07F01222D
:0B351E00300E07C20ED20F12353D2206
:0A353D00E5C120E5FBC2C4D2C5229F
:102F2200900374EBF0A3EAF0A3E9F090020AE070D8
:102F320002FF22900377E0FE6005D3941040037FE6
:082F4200002212328AEF604EFA
:102F4A00E4900379F0900377E0FF900379E0FEC301
:102F5A009F5024900374E0FBA3E0FAA3E0F98E8269
:102F6A00758300121B3FFF1231DBEF7002FF2290C4
:102F7A000379E004F080CEE490020CF012351E9042
:0E2F8A000378E07003200FFD90020CE0FF22A0
:032F98007FFF2296
:0E29150090038DEBF0A3EAF0A3E9F0A3EDF040
:10292300E4FFD3900263E09400900262E064809439
:102933008050012253E6FE900208E0FEA3E0240F3C
:10294300F58274023EF583E0FF900208E475F0011E
:10295300121BA0FCE5F064404C7006900208F0A343
:10296300F0900204E004F07006900203E004F0E447
:10297300FE900390E0FDEEC39D5054EEC39F504F75
:10298300900208E0FCA3E0240FF58274023CF58377
:10299300E0FD90038DE0FBA3E0FAA3E0F98E8275DE
:1029A3008300ED121B7E900208E475F001121BA058
:1029B300FCE5F064404C7006900208F0A3F090022E
:1029C30004E004F07006900203E004F00E80A2EE2F
:1029D300C39F5029900208E475F001121BA0FCE587
:1029E300F064404C7006900208F0A3F0900204E0FB
:1029F30004F07006900203E004F00E80D2900263AC
:102A0300E024FFF0900262E034FFF043E60190031C
:0C2A130090E0FEEFC39E50028002AF0670
:012A1F002294
:10345A00D3900263E09400900262E064809480401A
:08346A00047F0180027F0022B3
:031A180002236E38
:10236E00C0E0C0F0C083C082C0D075D000C000C035
:03237E0006C0078F
:10238100C210E5C054FE121D5D245D08245D0A24BF
:10239100240C24240E24D61024D612242A222435D7
:1023A1002824352A242A2C242A2E2417C023D0C2DB
:1023B10023BBE023BBE2000024E1C20D900250E008
:1023C100F5C2C2C5C2C490024F74FFF00224E3906B
:1023D100024FE0FFB4FF12900251E0F5C2C2C5C244
:1023E100C490024FE4F00224E3900251E0FEEFC3F7
:1023F1009E501790024FE0FF04F074522FF582E4D3
:102401003402F583E0F5C20224E3D2C490020CE465
:10241100F0C20F0224E390020C74FDF0D2C5C2C4D5
:102421000224E390024F74FFF0D20DC2C4C2C1D2A4
:10243100C50224E3E5C26007900207E0B5C20E9031
:102441000202E4F0C2C5C2C4D2C10224E3C2C4C2C2
:10245100C1300D030224DBC2C50224E3900202E075
:102461007020E5C2F0E0FFC3900204E09F7480F8A1
:10247100900203E064809850031232AF900202E0B0
:1024810004F0900204E024FFF0900203E034FFF036
:1024910090020DE0FEA3E0240FF58274023EF58365
:1024A100E5C2F090020DE475F001121BA0FEE5F00B
:1024B10064404E700690020DF0A3F0900202E01409
:1024C100F0700E900263E004F07006900262E00486
:1024D100F0D2C1800DC2C4300D08C20DD2C5800238
:1024E100D21030101053C17F43C180C2C5C2C4C2D3
:0724F100C1C210C20FC2C0FE
:1024F800D007D006D000D0D0D082D083D0F0D0E0A2
:0125080032A0
:05356500E5C15420FF48
:01356A00223E
:0735570043C14053E6FE22D0
:10267B00900348E0FFA3E0FCA3E0FDA3E0FBA3E095
:10268B00FAA3E0F990031AE572F0E573A3F0900357
:06269B0050E090031CF06A
:1026A100900314EFF0A3ECF0A3EDF0A3EBF0A3EA99
:0426B100F0A3E9F0B9
:1026B50090031D7403F0A374E8F0E5C120E5FBD297
:1026C500C1C2C4D2C5E4FF9003AAF030C0FDE5C085
:1026D50054FE2440700302277824FE602424E2601F
:1026E5000924FE600524E2022780C2C5EF600302CB
:1026F5002786900314E025E044A0F5C27F03022756
:1027050086EFB4030A900315E0F5C27F058072EFEA
:10271500B4050B900315A3E0F5C27F068063EF6453
:1027250006703E90031CE0900317700FE0FBA3E4D6
:1027350075F001121BB6A9F0FA8008E0FBA3E0FAD8
:10274500A3E0F9121B26F5C290031BE024FFF090CD
:10275500031AE034FFF0E07002A3E070247F0780E5
:1027650020EFB40706D2C47F0980169003AA74052A
:10277500F0800E9003AA7402F080069003AA7401FB
:10278500F0EFB40904C2C080369003AAE0FE6406E7
:102795006012EEB4021690031D74FFF5F0121BA033
:1027A50045F06008D2C5E49003AAF0FF9003AAE0C3
:1027B5006008C2C5D2C4C2C08005C2C00226D0E529
:0427C500C120E5FB4F
:0127C90022ED
:1027CA0090032AEFF0A3ECF0A3EDF0A3EBF0A3EA59
:0427DA00F0A3E9F08F
:1027DE009003327403F0A374E8F0E5C120E5FBD258
:1027EE00C1C2C4D2C5E4FF9003AAF030C0FDE5C05B
:1027FE0054FE24C870030228BB24AE607A24CA702B
:10280E00030228C324FE603824E2600924FE60051A
:10281E0024E20228CBC2C5EF700F90032AE025E018
:10282E0044A0F5C27F030228D1EF640160030228A1
:10283E00D190032AE025E044A1F5C27F040228D1FD
:10284E00EFB4030A90032BE0F5C27F058075EFB459
:10285E00050B90032BA3E0F5C27F068066EFB4064E
:10286E0006D2C57F01805CEFB404047F02805490D1
:10287E0003AA7405F0804C90032DE0FBA3E475F0E1
:10288E0001121BB6A9F0FAE5C2121B6C900331E0DF
:10289E0024FFF0900330E034FFF0E07002A3E0700C
:1028AE00087F09C2C1D2C4801A7F0280169003AA83
:1028BE007406F0800E9003AA7402F080069003AAAC
:1028CE007401F0EFB40904C2C080369003AAE0FE92
:1028DE0064066012EEB4021690033274FFF5F01225
:1028EE001BA045F06008D2C5E49003AAF0FF900348
:1028FE00AAE06008C2C5D2C4C2C08005C2C0022709
:06290E00F9E5C120E5FB24
:0129140022A0
:102A2000900348EFF090034BEBF0A3EAF0A3E9F03A
:082A3000900349ECF0A3EDF066
:102A3800757400543FF575543F605CC374409575D8
:102A4800FFE49574FE90034EE0FCA3E0FDC39FEC09
:102A58009E50068C728D7380048E728F7312267B43
:102A68009003AAE060037F022290034AE02573F0F6
:102A7800900349E03572F0900350E0700B90034CDE
:102A8800E5728573F0121BA0C390034FE09573F0B5
:102A980090034EE09572F090034EE0F572A3E0F5D6
:102AA80073D3E5739400E57294004070E573944025
:102AB800E5729400501312267B9003AAE060037F0E
:102AC8000222E4F572F57380D8900348E0FFA3E092
:102AD800FCA3E0FDA3E0FBA3E0FAA3E0F990031A4E
:102AE800E4F074401226979003AAE060037F022264
:102AF80074C02573F57374FF3572F57290034AE05C
:102B08002440F0900349E03400F0900350E07091C5
:0E2B180090034C75F040121BA0022AA97F000A
:012B2600228C
:10347200900330E4F0A304F01227CA9003AAE0609C
:07348200037F01227F0022FD
:1033F4009003A9EBF07B017A0379A990034EE4F0E2
:0A340400A304F0E4A3F0122A202232
:1032F400C007900369E0FFA3E0900330CFF0A3EF91
:10330400F0D0071227CA9003AAE060037F01227F4E
:02331400002295
:10340E00C007900371E0FFA3E090034ECFF0A3EF4F
:0A341E00F0E4A3F0D007122A2022E8
:0E316100900381EBF0A3EAF0A3E9F0A3EDF0F8
:10316F00E4900386F0900381E0FBA3E0FAA3E0F97B
:10317F00A3E0900377F0900385E0900378F0E4FFED
:10318F00122F22EFB4FF0D900386E0FE04F0EEC382
:06319F00940340D17E0004
:0131A5002207
:0B320F009003A1EBF0A3EAF0A3E9F0AC
:10321A007E007F007D10121D839003A1E0FBA3E0D6
:10322A00FAA3E0F97D10122915EF7002FF227F013F
:01323A002271
:10306F009003347422F0A3EFF0A37413F0121B2615
:10307F00900337F0900001121B3F900338F090003F
:10308F0002121B3F900339F0900003121B3F900375
:10309F003AF0900004121B3F90033BF09000051292
:1030AF001B3F90033CF0900006121B3F90033DF036
:1030BF007B017A037934E4900385F07D0A02316154
:103316009003917422F0A3EFF0A37403F0A374FF5B
:10332600F07B017A037991E4900385F07D04023104
:013336006135
:103337009003957422F0A3EFF0A3741CF0A374FF1D
:10334700F07B017A037995E4900385F07D040231DF
:013357006114
:10339900E4900399F0A3EFF0A3740AF0A3EFF07B94
:0F33A900017A037999E4900385F07D0402316184
:10335800A2AFE433FCC2AF758F0175B7A575B7F19D
:103368008F828E83EDF0E4F58FAF04EF24FF92AFE8
:013378002232
:10337900A2AFE433FDC2AF758F0375B7A575B7F179
:0F3389008F828E83E4F0F58FAF05EF24FF92AFB4
:013398002212
:1030CF0090039DEEF0A3EFF0A3ECF0A3EDF0EB4A2D
:1030DF00603990039DE0FEA3E0FFA3E0FCA3E0F5C1
:1030EF00828C83E0FD123358EB1B70011A9003A002
:1030FF00E004F0700690039FE004F090039EE0045C
:0C310F00F070CB90039DE004F080C32220
:08354F00E4900000F0A3F0225B
:10326400900000E0FEA3E0FF123379900000E0FE3E
:10327400A3E0FF7C007D027B007A021230CFE49051
:063284000000F0A3F0229F
:0A2D9700A905900387EEF0A3EFF00A
:102DA100EE54FEFE900000E0FCA3E0FD7002EE6C2C
:102DB1006057ED4C6003123264900387E0FEEE54DD
:102DC100FEFE7F00900000F0A3EFF0900389EEF08B
:102DD100A3EFF0A37400F0A37402F07E02900389C4
:102DE100E475F001121BB685F082F583E493FD9042
:102DF100038BE475F001121BB685F082F583EDF0CB
:102E0100EF1F70011EEF4E70D4900387E0FCA3E02A
:102E1100FDEC5401FC74022DF58274003CF583E94C
:012E2100F0C0
:012E2200228D
:10311B0090037AEEF0A3EFF0A3EBF0A3EAF0A3E9B0
:10312B00F090037F74FFF5F0121BB645F06026900C
:10313B00037AE475F001121BB6AFF0FE90037CE04E
:10314B00FBA3E475F001121BB6A9F0FA121B26FDC6
:06315B00122D9780CC222A
:0515430090031FEFF012
:10154800C20825E02425F8E6FE08E6FF900306EE2B
:10155800F0A3EFF0ED25E0244DF8E6FA08E6C39F86
:10156800FFEA9E900320F0A3EFF030095CC39003DC
:1015780020E064809480503890031FE0FF25E02429
:1015880039F8E6FA08E64A700BEF25E02439F876D0
:101598000008760390031FE0FF25E02439F808E6E9
:1015A80016187001161486024A6003021677805DC9
:1015B800D3900321E09404900320E0648094804059
:1015C80005C20902164D02166AD3900321E0940061
:1015D800900320E064809480405890031FE0FF252A
:1015E800E02439F8E6FA08E64A700BEF25E02439DA
:1015F800F8760008760390031FE0FF25E02439F809
:1016080008E616187001161486024A7062EF25E083
:101618002439F87600087601ED25E0244DF8E6FC3B
:1016280008E6FDEF25E02425F8A60408A605D2085B
:10163800803DC3900321E094FC900320E0648094F3
:101648007F501FD209ED25E0244DF8E6FE08E6FF9D
:1016580090031FE025E02425F8A60608A607D2086F
:10166800800D90031FE025E02439F8E4F608F62001
:10167800080302197A90031FE0FD25E0240AF8E622
:10168800FE08E67806C333CE33CED8F9FFED25E061
:1016980024F2F582E43402F583E04EFEA3E04FFF26
:1016A800E4FCFD900322121D20900320E0FEA3E03D
:1016B800FFD39400EE6480948050030217DDEE336C
:1016C80095E0FDFC7810121D0D900326121D209048
:1016D8000326E0FCA3E0FDA3E0FEA3E0FFC006C0F4
:1016E80007900306E0FEA3E0FFC374FF9FFF7403A7
:1016F8009EAB07FAE4F9F8D007D006121C579003FE
:1017080026121D20900326E0F8A3E0F9A3E0FAA32F
:10171800E0FBC00090031FE025E0240AF8E6FE087D
:10172800E6FFC374FF9FFF74039EFEE4FCFDD00038
:10173800121BCC900326121D2090031FE025E024E5
:101748000AF8E6FE08E6FFD3900307E09F90030639
:10175800E09E900326E0FCA3E0FDA3E0FEA3E0FFEB
:10176800E440047B5080027B30FAF9F8121BCC90DD
:101778000326121D20900322E0F8A3E0F9A3E0FA63
:10178800A3E0FBC000A3E0FCA3E0FDA3E0FEA3E010
:10179800FF7810121CFAD000EB2FFFEA3EFEE93D5D
:1017A800FDE83CFC900322121D20E47FFF7EFFFD34
:1017B800FC900322E0F8A3E0F9A3E0FAA3E0FBD34E
:1017C800121CE950030218FF900322121D2C00007E
:1017D800FFFF0218FF900320E0FEA3E0FFC3E49F91
:1017E800FFE49EFE3395E0FDFC7810121D0D90037A
:1017F80026121D20900326E0FCA3E0FDA3E0FEA333
:10180800E0FFC006C007900306E0FEA3E0FBAA06BF
:10181800E4F9F8D007D006121C57900326121D20B1
:10182800900326E0F8A3E0F9A3E0FAA3E0FBC000E8
:1018380090031FE025E0240AF8E6FE08E6FFE4FC32
:10184800FDD000121BCC900326121D2090031FE030
:1018580025E0240AF8E6FE08E6FFC3900307E09FA8
:10186800900306E09E900326E0FCA3E0FDA3E0FEC3
:10187800A3E0FFE450047B5080027B30FAF9F812B1
:101888001BCC900326121D20900322E0FCA3E0FD50
:10189800A3E0FEA3E0FFC004C005C006C007A3E0A4
:1018A800FCA3E0FDA3E0FEA3E0FF7810121CFAA859
:1018B80004A905AA06AB07D007D006D005D004C3F3
:1018C800EF9BFFEE9AFEED99FDEC98FC9003221237
:1018D8001D20E47FFF7EFFFDFC900322E0F8A3E0DB
:1018E800F9A3E0FAA3E0FBD3121CE9400A90032213
:1018F800121D2C00000000900322A3A3E0FEA3E029
:10190800FF90031FE0FB25E024F2F582E43402F5A2
:1019180083EEF0A3EFF0900322E0FCA3E0FDA3E048
:10192800FEA3E0FF7806121CFA900322121D20EB9A
:1019380025E0240AF8E6FE08E6FFE4FCFD90032211
:10194800E0F8A3E0F9A3E0FAA3E0FBC3121CE96006
:1019580021900322A3A3E0FEA3E0FF90031FE0254C
:10196800E0240AF8A60608A607E524452370031212
:0219780033D664
:01197A00224A
:04306A004102F1002E
:06356B00E49002F1F022E1
:07355E009002F17401F0225C
:102F9B009003A47404F0E4A3F0A3F012354F7E3930
:102FAB007F007B017A0379A490037FE4F0A304F004
:102FBB0012311BE49003A5F09003A5E0FFC3941E10
:102FCB00502A75F016EFA42401F582E5F03439AFE1
:102FDB0082FE7B007A00790890037FE4F0A37416DD
:102FEB00F012311B9003A5E004F080CC7E3B7F9563
:102FFB007B017A0379A690037FE4F0A304F01231EE
:04300B001B0232640E
:1033D60020111A3003133087129002F1E0700C901E
:0E33E600029FE0FF1233168002D287D211221E
:10342800903B95E493F46009903900E49364046058
:0A34380003122F9BE49002DAF02249
:10323B009002DAE0FFC3941E501EEF75F016A42423
:10324B0001F9743935F0FA7BFF78087C007D007E3C
:09325B00007F16121B00C21122B3
:1031A6009002DAE0C3941E502B12354F9002DAE0FB
:1031B60075F016A42401F582E5F03439AF82FE7B62
:1031C600007A00790890037FE4F0A37416F01231B8
:0531D6001B123264220F
:063571001231A6C2112276
:052CE300900309EDF073
:102CE80090030BE004F090030EEFF0A3EBF09003D9
:102CF80009E0FF90030EE0FED39F4003022D967576
:102D0800F016EEA42401F582E5F03439AF82900381
:102D180010F0A3EFF090030FE075F016A42401F56E
:102D280082E5F03439AF82900312F0A3EFF0E4901B
:102D3800030CF0A3F0900312E475F001121BB6AF78
:102D4800F0FE900310E0FCA3E0F5828C83E493FD91
:102D5800122D97900311E004F07006900310E00420
:102D6800F090030DE004F0700690030CE004F0C34B
:102D780090030DE0941690030CE0940040B71232D3
:0E2D88006490030EE004F0A3E004F0022CF6C9
:012D9600221A
:05250900900351EDF00C
:10250E00900356EFF0A3EBF0900351E0FF900356CB
:10251E00E0D39F400302267AA3E075F016A42401AF
:10252E00F582E5F03439AF82900352F0A3EFF0E478
:10253E00900358F0A3F0900358E0FEA3E0FFC3947D
:10254E0016EE94005038900352E0FCA3E0F5828C16
:10255E0083E493FD74DB2FF582E43402F583EDF012
:10256E00900353E004F07006900352E004F09003E1
:10257E0059E004F070C0900358E004F080B8900366
:10258E0056E075F016A42401F582E5F03439AF82D9
:10259E00900354F0A3EFF0900357E075F016A424C7
:1025AE0001F582E5F03439AF82900352F0A3EFF0DB
:1025BE00E4900358F0A3F0900352E475F001121B5F
:1025CE00B6AFF0FE900354E0FCA3E0F5828C83E4FA
:1025DE0093FD122D97900355E004F070069003546E
:1025EE00E004F0900359E004F07006900358E00404
:1025FE00F0C3900359E09416900358E0940040B74E
:10260E00900356E075F016A42401F582E5F03439F6
:10261E00AF82900354F0A3EFF0E4900358F0A3F0D0
:10262E00900358E0FCA3E0FDC39416EC9400502CEC
:10263E00900354E475F001121BB6AFF0FE74DB2D5F
:10264E00F582E43402F583E0FD122D97900359E0F4
:10265E0004F070CC900358E004F080C41232649001
:0C266E000356E004F0A3E004F00225167F
:01267A00223D
:0B2C2D0090033EEFF0A3EDF0A3EBF0EE
:102C3800A2AFE433A3F0C2AF12355790033FE0FED2
:102C480090033EE0FDEDFF900346EEF0A3EFF0E4C5
:102C5800900342F0900340E0FF900346E0FCA3E0BD
:102C6800FD7B017A0279DB900369E4F0A37416F026
:102C78001232F4900347E02416F0900346E0340043
:102C8800F0900342E075F016A42401F9743935F088
:102C9800FAA374FFF0A3EAF0A3E9F012354F90030A
:102CA80043A3E0FAA3E0AE02FF7B017A0279DB904E
:102CB800037FE4F0A37416F012311B123264900300
:102CC80042E004F0E0C3941E408A90029FE0FF12A5
:0A2CD80034EF900341E024FF92AFB7
:012CE20022CF
:0B197B0090035AEFF0A3EDF0A3EBF097
:10198600A2AFE433A3F0C2AF12355790035BE0FE7B
:1019960090035AE0FDEDFF90035FEEF0A3EFF0E455
:1019A60090035EF090035EE0FFC3941E504C75F00A
:1019B60016EFA42401F582E5F03439AF82FE9003D8
:1019C60061F0FAA3EFF0FB90035CE0FF90035FE0A9
:1019D600FCA3E0FDA9037BFF900371E4F0A374165A
:1019E600F012340E900360E02416F090035FE034AA
:1019F60000F090035EE004F080AA90029FE0FF12E0
:0A1A060034EF90035DE024FF92AF7F
:011A100022B3
:03000000020800F3
:03000300021A03DB
:03000B00021A06D0
:03001300021A09C5
:03001B00021A0CBA
:03002300021A0FAF
:03002B00021A12A4
:03003300021A1599
:03003B00021A188E
:03004300021A1B83
:03004B00021A1E78
:03005300021A216D
:03005B00021A2462
:03006300021A2757
:03006B00021A2A4C
:03007300021A2D41
:10080000E4F5D9E5EF7480F5FF7402F5EF787FE445
:10081000F6D8FD9000007F007E04E4F0A3DFFCDE4C
:07082000FA75817502086200
:100827000220D2E493A3F8E493A34003F68001F2F5
:1008370008DFF48029E493A3F85407240CC8C333D2
:10084700C4540F4420C8834004F456800146F6DFA1
:10085700E4800B010204081020408090300FE47EF2
:10086700019360BCA3FF543F30E509541FFEE49396
:10087700A360010ECF54C025E060A840B8E493A35D
:10088700FAE493A3F8E493A3C8C582C8CAC583CA88
:10089700F0A3C8C582C8CAC583CADFE9DEE780BE40
:01306E000061
:101A3000E709F608DFFA8046E709F208DFFA803E98
:101A400088828C83E709F0A3DFFA8032E309F60885
:101A5000DFFA8078E309F208DFFA807088828C83ED
:101A6000E309F0A3DFFA806489828A83E0A3F608A1
:101A7000DFFA805889828A83E0A3F208DFFA804C7B
:101A800080D280FA80C680D4806980F28033801052
:101A900080A680EA809A80A880DA80E280CA8033BB
:101AA00089828A83ECFAE493A3C8C582C8CCC58333
:101AB000CCF0A3C8C582C8CCC583CCDFE9DEE78003
:101AC0000D89828A83E493A3F608DFF9ECFAA9F082
:101AD000EDFB2289828A83ECFAE0A3C8C582C8CCD8
:101AE000C583CCF0A3C8C582C8CCC583CCDFEADEF1
:101AF000E880DB89828A83E493A3F208DFF980CC53
:101B000088F0EF60010E4E60C388F0ED2402B4044B
:101B10000050B9F582EB2402B4040050AF232345F2
:061B20008223901A80737D
:101B2600BB010689828A83E0225002E722BBFE02BD
:091B3600E32289828A83E49322F0
:101B3F00BB010CE58229F582E5833AF583E022505B
:101B4F0006E92582F8E622BBFE06E92582F8E222A5
:0D1B5F00E58229F582E5833AF583E49322BF
:101B6C00BB010689828A83F0225002F722BBFE0158
:021B7C00F32252
:101B7E00F8BB010DE58229F582E5833AF583E8F09D
:101B8E00225006E92582C8F622BBFE05E92582C849
:021B9E00F22231
:101BA000C5F0F8A3E028F0C5F0F8E58215827002D0
:061BB0001583E038F0226D
:101BB600A3F8E0C5F025F0F0E582158270021583E2
:061BC600E0C838F0E8223F
:101BCC00E88FF0A4CC8BF0A42CFCE98EF0A42CFCB8
:101BDC008AF0EDA42CFCEA8EF0A4CDA8F08BF0A436
:101BEC002DCC3825F0FDE98FF0A42CCD35F0FCEB95
:101BFC008EF0A4FEA9F0EB8FF0A4CFC5F02ECD395A
:0F1C0C00FEE43CFCEAA42DCE35F0FDE43CFC22C6
:101C1B0075F008758200EF2FFFEE33FECD33CDCC80
:101C2B0033CCC58233C5829BED9AEC99E582984003
:101C3B000CF582EE9BFEED9AFDEC99FC0FD5F0D6E0
:101C4B00E4CEFBE4CDFAE4CCF9A88222B800C1B90A
:101C5B000059BA002DEC8BF084CFCECDFCE5F0CB48
:101C6B00F97818EF2FFFEE33FEED33FDEC33FCEB81
:101C7B0033FB10D703994004EB99FB0FD8E5E4F93C
:101C8B00FA227818EF2FFFEE33FEED33FDEC33FC29
:101C9B00C933C910D7059BE99A4007EC9BFCE99A1D
:101CAB00F90FD8E0E4C9FAE4CCFB2275F010EF2F62
:101CBB00FFEE33FEED33FDCC33CCC833C810D70762
:101CCB009BEC9AE899400AED9BFDEC9AFCE899F89D
:0E1CDB000FD5F0DAE4CDFBE4CCFAE4C8F92230
:101CE900EB9FF5F0EA9E42F0E99D42F0E89C45F051
:011CF90022C8
:101CFA00E8600FECC313FCED13FDEE13FEEF13FFC8
:031D0A00D8F122EB
:101D0D00E8600FEFC333FFEE33FEED33FDEC33FC34
:031D1D00D8F122D8
:0C1D2000ECF0A3EDF0A3EEF0A3EFF02236
:101D2C00A8828583F0D083D082121D43121D4312EA
:101D3C001D43121D43E473E493A3C583C5F0C5830F
:101D4C00C8C582C8F0A3C583C5F0C583C8C582C801
:011D5C002264
:101D5D00D083D082F8E4937012740193700DA3A315
:101D6D0093F8740193F5828883E473740293686029
:061D7D00EFA3A3A380DF29
:101D8300EF4E6012EF60010EEDBB010B89828A8377
:101D9300F0A3DFFCDEFA2289F05007F709DFFCA984
:0C1DA300F022BBFEFCF309DFFCA9F022DB
:00000001FF
